:100000000C9455040C949C040C949C040C949C0437
:100010000C949C040C949C040C949C040C949C04E0
:100020000C949C040C949C040C9493260C946527CB
:100030000C941D1F0C949C040C949C040C949C0424
:100040000C949C040C949C040C949C040C949C04B0
:100050000C944A0B0C94911F0C949C040C949C04DB
:100060000C949C040C949C040C949C040C949C0490
:100070000C949C040C949C040C949C040C949C0480
:100080000C949C040C949C040C949C040C949C0470
:100090000C949C040C949C040C949C040C949C0460
:1000A0000C949C040C949C040C949C04FB14FB1472
:1000B0002D152D157A15981505170517DA157316D0
:1000C000841684160517E4168B178B179D179D173A
:1000D00094179D179D179D178B178B1799179D17B1
:1000E0009D179917D227F927F128F927F1284528D4
:1000F0006828F128BF28CE2820202020202020009A
:100100005343524C434B200020202020202020002D
:100110004341504C434B2000202020202020200031
:100120004E554D4C434B2000556E646566696E65B7
:100130006400464E0A0044656661756C740A004CA2
:10014000617965723A20004B0052004E0050005118
:10015000004F000151A800BF5C4A00B2004D00C032
:100160005C2900A6000100AE00005C000000000059
:1001700000000000000001010203040506080A0C4B
:100180000F1114181C2024292E33393F464C535B81
:10019000626A7179818A929AA2AAB2B9C1C8CFD58E
:1001A000DCE1E7EBF0F4F7FAFCFDFEFFFEFDFCFA04
:1001B000F7F4F0EBE7E1DCD5CFC8C1B9B2AAA29A57
:1001C000928A8179716A625B534C463F39332E299A
:1001D00024201C1814110F0C0A0806050403020140
:1001E000010000000000000000000000AE00AF00B1
:1001F000DA02818FD9F1DB40A4A62EAF00A0C000A7
:10020000A1C800AED580A81FD300408D14200000E7
:1002100000000000003E5B4F5B3E003E6B4F6B3EBC
:10022000001C3E7C3E1C00183C7E3C18001C577D88
:10023000571C001C5E7F5E1C0000183C180000FF6D
:10024000E7C3E7FF00001824180000FFE7DBE7FF23
:100250000030483A060E00262979292600407F05FD
:10026000050700407F05253F005A3CE73C5A007FC8
:100270003E1C1C0800081C1C3E7F0014227F221418
:10028000005F5F005F5F0006097F017F00006689F5
:10029000956A0060606060600094A2FFA29400080C
:1002A000047E04080010207E20100008082A1C0884
:1002B00000081C2A0808001E10101010000C1E0C4C
:1002C0001E0C0030383E383000060E3E0E06000090
:1002D000000000000000005F0000000007000700B1
:1002E00000147F147F1400242A7F2A12002313088D
:1002F00064620036495620500000080703000000E1
:100300001C224100000041221C00002A1C7F1C2AE4
:100310000008083E08080000807030000008080847
:100320000808000000606000002010080402003E81
:100330005149453E0000427F40000072494949460C
:10034000002141494D33001814127F100027454504
:100350004539003C4A49493100412111090700361D
:100360004949493600464949291E00000014000049
:10037000000040340000000008142241001414144E
:100380001414000041221408000201590906003E1D
:10039000415D594E007C1211127C007F494949365B
:1003A000003E41414122007F4141413E007F494999
:1003B0004941007F09090901003E41415173007F15
:1003C0000808087F0000417F4100002040413F01B4
:1003D000007F08142241007F40404040007F021C03
:1003E000027F007F0408107F003E4141413E007FB4
:1003F00009090906003E4151215E007F091929467D
:100400000026494949320003017F0103003F404073
:10041000403F001F2040201F003F4038403F006306
:1004200014081463000304780403006159494D4320
:1004300000007F41414100020408102000004141BA
:10044000417F00040201020400404040404000009F
:1004500003070800002054547840007F28444438A3
:1004600000384444442800384444287F0038545419
:1004700054180000087E09020018A4A49C78007F8C
:10048000080404780000447D4000002040403D0006
:10049000007F102844000000417F4000007C047869
:1004A0000478007C0804047800384444443800FC94
:1004B000182424180018242418FC007C08040408BC
:1004C0000048545454240004043F4424003C404059
:1004D000207C001C2040201C003C4030403C00445C
:1004E00028102844004C9090907C004464544C4464
:1004F000000008364100000000770000000041368F
:100500000800000201020402003C2623263C0000F1
:100510000000000000404040F0F8F8FF38FFF8F815
:100520003FF8F8FF38FFF8F8F040404000000000C6
:10053000000080C0C0C0800000C0C08000000080FB
:10054000C0C000C0C0000080C0C00000000000C0EB
:10055000C0C0C0C000C0C00000000000000000001B
:10056000000000000000000000000000000000008B
:10057000000000000000000000000000000000007B
:100580000000000000000000000000000000C0F0BB
:10059000F8FC3E1E06010000007F4141417F007FC4
:1005A0004141417F000080C0E07E5B4F5BFEC000A8
:1005B00000C000DCD7DEDEDED7DC00C000000000BB
:1005C000000000000000000000000000000000002B
:1005D0000000000000494949FFFFFFFFE0DFBFBF07
:1005E00000BFBFDFE0FFFFFFFF49494900000000F7
:1005F000001F3F6060E0BF1F007F7F071E381E079F
:100600007F7F007F7F0E1F3B716000000000007F36
:100610007F0C0C0C007E7E007F7E0303007F7E0338
:10062000037E7E03037F7E000F3E703C063C703EDF
:100630000F00327B49493F7E007F7E0303001E3F4F
:1006400069696F2600000000000000000000030F31
:100650001F3F3C7870600000007F4141417F007F78
:100660004141417F00307B7F7830202030787F3BD4
:100670000003000F7F0F0F0F7F0F0003000000002B
:10068000000000000000000000000000000000006A
:100690000000000000010101070F0F7F0F7F0F0F07
:1006A0007E0F0F7F0F7F0F0F070101010000000079
:1006B0000000000000000101000000000000000038
:1006C000000000000000000000000000000000002A
:1006D000000000000000000000000000000000001A
:1006E000000000000000000000000000000000000A
:1006F00000000000000000000000000000000000FA
:1007000000000000000000000000000000000000E9
:1007100000000000000000000000000000000000D9
:1007200000000000000000000000000000000000C9
:1007300000000000000000000000000000000000B9
:1007400000000000000000000000000000000004A5
:10075000033000000028035700610073006800693F
:10076000006E00670074006F006E0020004D006195
:1007700000630072006F00700061006400000012EE
:10078000036D00650072006C0069006E003000347B
:100790000000000403090409023B00020100A0FA62
:1007A00009040000010301010009211101000122D7
:1007B00040000705810308000A0904010001030045
:1007C0000000092111010001228500070582032094
:1007D000000A1201100100000008EDFE2A000100CD
:1007E0000102030105010902A10185020901A1001D
:1007F00005091901290515002501950575018102D5
:100800009501750381010501093009311581257FA5
:1008100095027508810609381581257F95017508AF
:100820008106050C0A38021581257F95017508811E
:1008300006C0C005010980A10185031A81002A8331
:1008400000160100260300950175108100C0050CFB
:100850000901A10185041A01002A9C021601002643
:100860009C02950175108100C005010906A10105D2
:100870000719E029E7150025019508750181029502
:1008800001750881010507190029FF150026FF00E1
:10089000950675088100050819012905950575015A
:1008A0009102950175039101C00011241FBECFEF85
:1008B000DAE0DEBFCDBF04B603FE27C080910F048F
:1008C00090911004A0911104B09112048730904BC4
:1008D000A740B04BD1F410920F0410921004109264
:1008E00011041092120414BE84B7877F84BF0FB620
:1008F000F894A895809160008861809360001092C0
:1009000060000FBEE0E0F8E3099511E0A0E0B1E07F
:10091000EAE0F4E502C005900D92AA33B107D9F7D9
:1009200024E0AAE3B1E001C01D92AF30B207E1F7C5
:100930000E94C2230C94032A0C940000CF93C62F6C
:100940006091C1017091C2018091C3019091C40175
:100950000E94831D882319F0813039F00EC0CC230A
:1009600011F089EA07C08AEA05C0CC2311F08BEAAE
:1009700001C08CEACF910C94A414CF910895CF9329
:1009800060E08FE391E00E948E0D6091C101709153
:10099000C2018091C3019091C4010E94831D8823EC
:1009A00031F0813051F460E082E391E003C060E017
:1009B00086E391E00E948E0D05C060E088E291E040
:1009C0000E94A00D0E94D111C82F80FD03C088E1B4
:1009D00091E002C080E291E060E00E948E0DC1FDD6
:1009E00003C088E091E002C080E191E060E00E94F5
:1009F0008E0DC2FD03C088EF90E002C080E091E060
:100A000060E0CF910C948E0D81E0089581E008950F
:100A10000C9406051F93CF93DF9300D000D01F9254
:100A2000CDB7DEB749835A836B8320917E018981DC
:100A30009A81211112C0662349F00E945E1C182F72
:100A4000682F89819A810E94071C03C00E94321C72
:100A5000182F69817A81812F04C00E945E1C6981F0
:100A60007A810F900F900F900F900F90DF91CF91A0
:100A70001F910C94DF05FC014081518162817381DB
:100A800084810C940A050E94D31D811102C00E942A
:100A90007C1E0E94B90B0E94D30B0C94A6080E94E6
:100AA000E30B0C94A20808950C94530581E008957B
:100AB0000C945605CF93C82F0E9454058C2F0E948A
:100AC0005805CF91089508950E9479170E946305F3
:100AD0002FEF84E39CE0215080409040E1F700C07C
:100AE00000000C94B71F0F931F93CF93DF938C01DB
:100AF0000E943B05EC01B8010E940805882309F417
:100B000058C0B801CE010E947B0F882309F451C060
:100B1000B801CE010E94BC0F882309F44AC0F80135
:100B200082818823A9F0C13C8CE5D80771F0CE3DC5
:100B3000ECE5DE0739F0C115FCE5DF0749F40E945A
:100B4000640537C00E947C1E34C00E94DC0931C09D
:100B5000C631DC4539F50E94DF1C982FF8018281EF
:100B60002091080130910901882379F09A7A81E077
:100B700009F480E080933A01911102C069E201C05A
:100B800065E3C9010E94B61E0AC080913A01811135
:100B900002C069E201C065E3C9010E94B81E0E945B
:100BA000201D07C0C801DF91CF911F910F910C94B8
:100BB000040580E0DF91CF911F910F910895272FB9
:100BC00030E0F901EE0FFF1F2E0F3F1FF90199E0F2
:100BD000899FE00DF11D1124E60FF11DEE0FFF1F9F
:100BE000E95BFE4F859194910895CF93DF930E9426
:100BF000DF050E94C107EC01811523E5920708F08B
:100C000058C0811542E5940708F028C18F3F91052F
:100C100009F0F8F4803F910508F016C1883A910573
:100C200070F4853A910508F0A5C08130910509F46A
:100C3000A4C108F455C1049708F09FC151C18F3B6E
:100C4000910508F4A2C0805E9109089708F495C147
:100C500047C1C11580E5D80758F4C11520E4D20773
:100C600008F0F4C0C11540E2D40708F486C138C1C9
:100C7000C11581E5D80708F0ECC0CE0174E0969567
:100C800087957A95E1F783709C2F937021E030E08F
:100C900002C0220F331F9A95E2F73C68382BCF70C1
:100CA000C695C69580E2C89FE0011124C22BD32BC4
:100CB00064C181152AE5920798F5811549E59407E5
:100CC00008F0F0C0C11585E5D807D8F4C11524E5B2
:100CD000D20708F0D8C0CE018370992721E030E018
:100CE00002C0220F331F8A95E2F78C2F86958695D6
:100CF00040E2849FC0011124E901C82BD92BDA6896
:100D00003CC1C11546E5D40708F4C2C0C11588E549
:100D1000D80708F4E5C0DC2FCC27C06FD06A2DC1FE
:100D20008E3B2CE5920709F4D2C070F4CC3B8CE5E5
:100D3000D80709F4C6C008F0C7C0CB3BDC4509F0B2
:100D4000CFC0C0E0D4ED19C1C03C8CE5D80709F490
:100D5000C4C008F4BFC0CE0190568115904208F07F
:100D6000BFC08D2F8F710E945508DD27D0628F7113
:100D7000D82B03C1853A910509F4B5C0863A91058F
:100D800009F0B4C0C2E8D0E4F8C0883A910509F48B
:100D9000B0C0893A910509F4AFC08A3A910509F4C7
:100DA000AEC08B3A910509F4ADC08C3A910509F4B7
:100DB000ACC08B3B910509F4ABC08C3B910509F4A9
:100DC000AAC08D3A910509F4A9C0803B910509F4A8
:100DD000A8C08E3A910509F4A7C08F3A910509F48D
:100DE000A6C0813B910509F4A5C0823B910509F499
:100DF000A4C0833B910509F4A3C0843B910509F489
:100E0000A2C0853B910509F4A1C0863B910509F478
:100E1000A0C0873B910509F49FC0883B910509F468
:100E20009EC0893B910509F49DC08D3B910509F455
:100E30009CC08E3B910509F49BC08A3B910509F447
:100E40009AC0C0E0D4E499C0D06597C0DF70D06A82
:100E500094C0DC2FCC27C16FD06A8FC083709927D4
:100E600021E030E002C0220F331F8A95E2F78C2F79
:100E70008695869540E2849FC0011124E901C82B24
:100E8000D92BDC687AC0DC2FCC27C46FD06A75C040
:100E90008C2F0E9455088F71C82FD0E0DC2FCC27F3
:100EA000D0626BC08F700E94550894E0D695C795AC
:100EB0009A95E1F7CF70D0E0DC2FCC27D069C82B12
:100EC0005CC0C0E0D5ED59C0C0E0D1ED56C0C0E077
:100ED000D0ED53C0C0E0D2ED50C0C0E0D3ED4DC066
:100EE000C0E0D0E04AC0C1E8D0E447C0C3E8D0E4E5
:100EF00044C0C2EED4E441C0C9EED4E43EC0CAEE60
:100F0000D4E43BC0C5EBD4E438C0C6EBD4E435C070
:100F1000C3EBD4E432C0C4EBD4E42FC0C7EBD4E4B9
:100F20002CC0CCECD4E429C0CDECD4E426C0C3E87A
:100F3000D5E423C0CAE8D5E420C0C2E9D5E41DC089
:100F4000C4E9D5E41AC0C1E2D6E417C0C3E2D6E4CE
:100F500014C0C4E2D6E411C0C5E2D6E40EC0C6E2B5
:100F6000D6E40BC0C7E2D6E408C0CFE6D4E405C09F
:100F7000C0E7D4E402C0CAE2D6E4CE01DF91CF914B
:100F800008958238910569F1B0F48133910509F42F
:100F90006DC048F48932910509F463C08A32910525
:100FA00009F469C008958533910509F455C0893362
:100FB0009105B9F00895833E910569F138F4803EBA
:100FC0009105B1F0823E910509F10895863E9105A3
:100FD000A9F1873E9105B9F1843E910509F064C0FD
:100FE00023C02091000420FD4FC021FD4DC0089575
:100FF0008091000480FD44C08091010480FF44C0C2
:101000008091000484FD42C083EE4DC080910004B5
:1010100082FF38C0F5CF8091000482FD33C08091FB
:10102000010480FD31C0ECCF8091010481FF32C00A
:101030008091000484FD2AC087EE35C080910004B1
:1010400083FF26C0F5CF8091000483FD21C08091ED
:10105000010481FD1FC0ECCF8091000485FD1CC000
:101060001DC08091000485FD19C016C08091000448
:1010700086FD16C017C08091000486FD13C010C005
:1010800089E311C082EE0FC080EE0DC080E00BC07E
:1010900086EE09C084EE07C089E205C085E303C07F
:1010A0008AE201C081E390E008959091000492FFEC
:1010B0000DC0282F2871283019F4877F846006C05E
:1010C000282F2471243011F48B7F886093FF0DC08A
:1010D000282F2871283119F4877E846106C0282FB3
:1010E0002471243111F48B7E88612091010420FF4A
:1010F0000DC0382F3871383019F4877F816006C0F1
:10110000382F3171313011F48E7F886021FF0DC08E
:10111000282F2871283119F4877E816106C0282F75
:101120002171213111F48E7E886194FD877E0895AE
:10113000E82FF0E0E051FE4F808108950895089572
:101140000C949F080C94A0080C949F080C94A4087D
:10115000CF93DF93AEE1B1E041E251E061E070E0B6
:101160008D91E82FE295EF70F0E021A18F70EB01F7
:1011700002C0CC0FDD1F8A95E2F7CE019C2F90951F
:10118000922391A392A1892B82A34A175B0741F76F
:10119000ABE1B1E04EE151E061E070E08D91E82F0C
:1011A000E295EF70F0E021A18F70EB0102C0CC0F4F
:1011B000DD1F8A95E2F7CE019C2F9095922391A393
:1011C00092A1892B82A34A175B0741F71092ED0188
:1011D0001092F0011092EE011092F1011092EF01C5
:1011E0001092F20183E00E948709DF91CF910C9465
:1011F00043055F926F927F928F929F92AF92BF92C0
:10120000CF92DF92EF92FF920F931F93CF93DF93D2
:101210006EE171E0ADEEB1E020EFA22E21E0B22E42
:10122000612C01E010E06D015C901C92EB01899152
:10123000BE01E82FE295EF70F0E021A18F70A801C8
:1012400002C0440F551F8A95E2F7CA01242B21A33F
:1012500022A1942E9094292122A350EA5A95F1F7C5
:101260009BE1E92E91E0F92E40E050E0E701899002
:101270007E01282D22952F7030E0E90128A17C9075
:1012800030E0D82DDF7002C035952795DA95E2F76A
:1012900020FD08C0302F042E01C0330F0A94EAF756
:1012A000232F01C020E027292C934F5F5F4F43304D
:1012B0005105E1F691A1992291A292A1892B82A3D5
:1012C000119681E0F6019081951101C080E0682AB5
:1012D000AA16BB0609F0A7CF262D43E060EF71E008
:1012E0008DEE91E00E9488090E944F05862DDF91C6
:1012F000CF911F910F91FF90EF90DF90CF90BF9013
:10130000AF909F908F907F906F905F900895089519
:10131000FF920F931F93CF93DF938C01F62ED72F5D
:10132000C42F222349F081E080933D010E944F1F8A
:1013300090933C0180933B0180913D018823C1F053
:1013400080913B0190913C010E94671F069780F0BD
:10135000EF2DFD2FD8014C2F50E0CD01801B910BBC
:10136000841795071CF48D918193F7CF10923D015E
:10137000DF91CF911F910F91FF9008958091F3011C
:1013800086958695869508958091F30181FD07C025
:1013900082608093F3010E94081E0C94350B08951F
:1013A0008091F30181FF07C08D7F8093F3010E943C
:1013B000081E0C94410B08958091F30181FD0C945B
:1013C000D0090C94C4098091F30186958170089529
:1013D0008091000108950E94D31D811102C00E94D6
:1013E0007C1E0E94041E8093F301282F26952695CB
:1013F000269530E02430310524F087708861809391
:10140000F3018091F30180FF04C08695869586954F
:1014100001C080E00C94120B2091F301822F86957D
:1014200086958695482F50E04330510554F48F5FE0
:10143000982F990F990F990F822F8770892B80937E
:10144000F3018091F30181608093F3010E94081EF3
:101450008091F3018695869586950C94120B809168
:10146000F301982F969596959695A1F0915E990F18
:10147000990F990F8770892B8093F301887F91E0F2
:1014800009F490E08091F30190FB80F98093F301DF
:101490000E94081E8091F3018695869586950C948E
:1014A000120B8091F30180FD13C081608093F301E2
:1014B000813019F489E08093F3018091F3010E9457
:1014C000081E8091F3018695869586950C94120BE3
:1014D00008958091F30180FF08C08E7F8093F3010F
:1014E0000E94081E80E00C94120B08958091F30175
:1014F00080FD0C94690A0C94510A9091F301892F94
:101500008695869586958F5F8F719770843038F4B5
:10151000880F880F880F892B8093F30102C0909366
:10152000F3018091F301887F91E009F490E08091CC
:10153000F30190FB80F98093F3010E94081E8091D3
:10154000F3018695869586950C94120B843008F0ED
:1015500083E09091F3019770282F220F220F220F22
:10156000922B9093F301987F21E009F420E0909171
:10157000F30120FB90F99093F3010C94120B0E945D
:10158000A60A8091F3010C94081ECF92DF92EF928D
:10159000FF928C3724E1920728F469E070E00E9402
:1015A000412929C0A0E0B0E08A50974DAF4FBF4F0E
:1015B0006627782F892F9A2F25EF38E241E050E0F7
:1015C0000E94692969017A01CA01B9010E9425298D
:1015D0009B01AC01C701B6010E942529BB27A92F99
:1015E000982F872F009721E0A207B10511F0BC01C9
:1015F00002C06FEF7FEFCB01FF90EF90DF90CF90B5
:101600000895E82FE295EF70F0E032A1282F2F70B7
:1016100081E090E001C0880F2A95EAF78095832346
:1016200082A30895843030F4811105C09091800028
:101630009F7D04C083E09091800090629093800031
:10164000282F30E0AFEFBFEF0E94912923E030E078
:1016500040E050E00E946929C9010E94C50A9093A8
:101660008B0080938A000895089510923F01109294
:101670003E0110924001EFE6F0E0808181608083BE
:101680000895EFE6F0E080818E7F80830E94BE099E
:101690000C94120B1F920F920FB60F9211242F93DE
:1016A0003F934F935F936F937F938F939F93AF93EA
:1016B000BF93CF93EF93FF930E94E80940913E01BF
:1016C00050913F014F5F5F4F94EF899F900111242C
:1016D000CA01B9010E94412990933F0180933E01C4
:1016E000B901660F672F661F770B71950E9441291C
:1016F0006F7780914001823019F4603451F404C056
:10170000813039F46F3729F480916F008E7F809398
:101710006F00E62FF0E0E559FE4FC4910E94BE092C
:10172000282F41E051E0C49FC001C59F900D1124B6
:1017300063E070E00E944129269FC001279F900D21
:1017400011240E94C50A90938B0080938A00FF9118
:10175000EF91CF91BF91AF919F918F917F916F91B9
:101760005F914F913F912F910F900FBE0F901F905F
:101770001895269A86E30E94010B82E280938000EE
:1017800089E1809381008FEF9FEF90938700809392
:1017900086000E94EB090E94E30981110C94350B2D
:1017A00008950C949E0454985C9A3E98469A89B188
:1017B00082958170369902C090E001C092E0892B39
:1017C000809343010895E0914301EE0FEE0FE09303
:1017D000430149B144FB882780F990E046B146FBBC
:1017E000222720F930E046FF02C022E030E0822BC1
:1017F000932B8E2B809343018F70E82FF0E0EF5DE9
:10180000FE4F908180914201890F80934201843084
:101810004CF0809141018F5F8093410161E080E055
:101820000E94D10B809142018D3F4CF48091410187
:1018300081508093410160E080E00E94D10B809153
:101840004201837887FF03C081508C6F8F5F809344
:1018500042010895EF92FF920F931F93CF93DF936E
:10186000EC017B0164E670E088E70E94ED108C01DA
:10187000EC0EFD1ECE15DF0561F017FD0AC0FE015E
:10188000849164E670E00E9444118C012196892BBA
:1018900089F30E94C811C801DF91CF911F910F9168
:1018A000FF90EF9008950895E4EFF1E080E092E07A
:1018B000DF019C011D9221503040E1F7F093F903C4
:1018C000E093F8038FEF9FEF9093700180936F0187
:1018D00008950E94530C80936B0180FD02C080E844
:1018E00001C080E280936A010E94E7106DE070E021
:1018F00082E092E00E942A0C892B11F080E008958A
:1019000080916B0163E070E081FD03C08FEF91E097
:1019100002C08CEF91E00E942A0C892B79F76DE0D0
:1019200070E08FEE91E00E942A0C892B39F70E941B
:101930005B1FDC01CB01805A9541AF4FBF4F8093B5
:10194000F4039093F503A093F603B093F7030E947A
:10195000540C81E080936E0180936D0110926C01B4
:10196000089520916A0136E0839FC0011124629F8F
:10197000800D911D1124811522E0920714F080E062
:1019800090E08C509E4F9093F9038093F803089554
:101990002091F8033091F9032E5E314040916A01A5
:1019A000642F70E0C9010E944129481B463010F4A1
:1019B000240F311D211582E0380710F020E030E0BF
:1019C0002C503E4F3093F9032093F8030895CF93A2
:1019D000DF938A3011F481E003C08D3029F480E078
:1019E000DF91CF910C945D0DC62F682F8091F80385
:1019F0009091F90326E0FC01A4E4B1E001900D927E
:101A00002A95E1F7613E30F026E0FC0111922A951B
:101A1000E9F70AC0F6E06F9FB0011124615F7D4FC6
:101A200046E050E00E94AB29C11135C0C091F803D7
:101A3000D091F90346E050E0BE0184E491E00E94B9
:101A4000B429892BB1F1C45FD1409E0185E0369560
:101A500027958A95E1F781E090E0AC0102C0440F40
:101A6000551F2A95E2F720916F0130917001242BC8
:101A7000352B269645E0D695C7954A95E1F702C0E5
:101A8000880F991FCA95E2F7822B932B90937001D0
:101A900080936F010EC0E091F803F091F9039F016C
:101AA0002A5F3F4F2E173F0709F28081809581936F
:101AB000F9CFDF91CF910C94C80CCF93E82F2091F0
:101AC000F8033091F903245F314040916A01642F9B
:101AD00070E0C9010E944129481B842FEE2359F070
:101AE00066E00E943529C82FC150B0F060E080E266
:101AF0000E94E70CF9CFA901480F511D4115524032
:101B000018F080E020E030E0280F311D2C503E4FCF
:101B10003093F9032093F803CF9108951F93CF9347
:101B2000DF93EC01162FFE018491882329F0612FA9
:101B30000E94E70C2196F7CFDF91CF911F91089576
:101B40000E948E0D81E00C945D0D0E945B1FDC01F4
:101B5000CB01805A9541AF4FBF4F8093F4039093D0
:101B6000F503A093F603B093F70380916D01811103
:101B70000BC062E070E08DEE91E00E942A0C892B90
:101B800019F481E080936D0180916D0108956F9249
:101B90007F928F929F92AF92BF92CF92DF92EF92FD
:101BA000FF920F931F93CF93DF9320916F0130919A
:101BB00070012115310509F4D4C080916C018111A7
:101BC000D0C061E070E0082F10E03B01082E02C099
:101BD000660C771C0A94E2F7A30142235323452B9A
:101BE00011F48F5FF0CF90916B01980165E0220FA7
:101BF000331F6A95E1F790FD12C08295880F8076B9
:101C000080930301220F232F221F330B3195209342
:101C10000601815E809304011092070112C045E025
:101C2000369527954A95E1F7220F220F220F209330
:101C3000030110920601295F2093040183E0809341
:101C4000070124E630E047E050E061E071E088E71A
:101C50000E947411892B09F084C080916B0180FD72
:101C600023C0A80195E0440F551F9A95E1F74C5009
:101C70005E4F04E610E020E230E060E488E70E9476
:101C80009B11892B09F06DC00E94A50DE301C09541
:101C9000D09580916F0190917001C823D923D09382
:101CA0007001C0936F015DC080E2EAE4F1E0DF0102
:101CB0001D928A95E9F785E0000F111F8A95E1F7DB
:101CC000A5E3B1E041E351E0992493942D91EA0119
:101CD0008991AE01B801680F711D6C507E4F30E0E4
:101CE000265B3E4FF90197E07F01E21AF30AA92C27
:101CF00001C0AA0CEA94EAF77B01B12CE7018991B3
:101D00007E018A21892E8B18D82DD770CD2E0D2ECD
:101D1000000CDD08C82F01C0CC0FDA95EAF7D1948A
:101D2000C194D108D7E0CD22DD2401C08695CA94A4
:101D3000EAF78C2BD0808D298083B39488E0B81289
:101D4000DDCF915031969F3F79F6C1E0A933BC07B2
:101D500009F0BCCF04E610E020E230E04AE451E0B4
:101D60008CCFDF91CF911F910F91FF90EF90DF907B
:101D7000CF90BF90AF909F908F907F906F9008957D
:101D800080916D01882369F062E070E08BEE91E054
:101D90000E942A0C892B19F080916D0108951092F0
:101DA0006D0190916D0181E089270895CF92DF92B6
:101DB000EF92FF9280916E01882321F160E080E034
:101DC0000E94B10C0E94BF040E94C70D80916D015A
:101DD0008823C1F0C090F403D090F503E090F6039F
:101DE000F090F7030E945B1FDC01CB018C199D0969
:101DF000AE09BF09B7FD06C0FF90EF90DF90CF900E
:101E00000C94C00EFF90EF90DF90CF9008950F9349
:101E10001F93CF93DF93C62FD42F122FFC01828103
:101E20008823C9F0609373010E944F1F9093720141
:101E30008093710180E28C0F883008F057C0C77022
:101E400081E001C0880FCA95EAF7DF91CF911F9119
:101E50000F910C94B71480917301681330C0809176
:101E60007101909172010E94671F883C910538F5BD
:101E700000E20D0FCD17B9F080E28C0F883040F4EE
:101E8000C77081E001C0880FCA95EAF70E94BE14AE
:101E9000083028F581E09D2F977001C0880F9A9532
:101EA000EAF70E94B714812F0E94A4140830F0F4BE
:101EB000D77081E001C0880FDA95EAF70AC080E2A6
:101EC0008C0F883098F4C77081E001C0880FCA95E4
:101ED000EAF7DF91CF911F910F910C94BE14812FDF
:101EE000DF91CF911F910F910C94A414DF91CF91AA
:101EF0001F910F9108959C01CB01233F4CE53407BE
:101F0000F9F078F4283DFCE53F07B9F0293D4CE5B0
:101F1000340711F1273D3C4531F526E241EE61EEF3
:101F20001EC0253FFCE53F0799F070F0263F3C4579
:101F3000D1F427E245EE66EE12C027E245EE0EC070
:101F400026E241EE60EE0BC027E245EE64EE07C0EC
:101F500026E241EE62EE03C028E241E065EE0E9417
:101F6000070F80E00895FC018281882319F0109208
:101F70007301089581E00895CF93DF93EC01FB0195
:101F80008281882309F41FC1C230FCE5DF0708F411
:101F90001BC1C6319CE5D90738F09E012A5F3C453C
:101FA0002930310508F010C10E94E61D909301040C
:101FB00080930004C031ECE5DE0709F4C3C008F0EB
:101FC00041C0C8308CE5D80709F49AC0F0F4C43099
:101FD000ECE5DE0709F487C068F4C2308CE5D80769
:101FE00009F477C0C330DC4509F0E3C080910004F8
:101FF000826076C0C630ECE5DE0709F46EC008F0FA
:102000007BC08091000488606BC0CC308CE5D80721
:1020100009F485C068F4CA30ECE5DE0709F474C041
:1020200008F079C00E94791780910004806858C038
:10203000CE308CE5D80709F476C008F07FC08091D7
:1020400000048BC0CB3FECE5DE0709F44FC018F568
:10205000C3318CE5D80709F47DC078F4C131ECE5D3
:10206000DE0709F473C0C231DC4509F0A2C00E944A
:102070007917809100048F7733C0C5318CE5D8077C
:1020800009F472C008F486C0CA3FDC4509F091C06B
:10209000809101043EC0CF3FFCE5DF0709F45FC03B
:1020A00058F4CD3F9CE5D90709F444C008F43FC07B
:1020B0008091010482602DC0C130FDE5DF0709F485
:1020C00075C008F45DC0C230DD4509F072C080E023
:1020D0006EC080910004816003C080910004806123
:1020E0008093000466C08091000411C080910104B7
:1020F0008260809301045DC0809100048062F0CF13
:10210000809100048064ECCF80910004886084603A
:10211000E7CF8160EECF809100048E7FE1CF809188
:1021200000048D7FDDCF80910004877FD9CF80911F
:10213000010418C0809101048D7FDBCF80910004E1
:102140008F7ECECF809100048F7DCACF8091000416
:102150008F7BC6CF80910004877F8B7FC1CF80911A
:1021600001048D7F8E7FC5CF8091000482FB2227E2
:1021700020F991E0922790FB82F990FB83F9B0CF90
:1021800080910104982F909591708E7F892B90FB00
:1021900081F9AFCF0E9479178091000487FB222735
:1021A00020F991E0922790FB87F99ACF81E00E9475
:1021B0007E1E80910004909101040E94F71D0E94F0
:1021C000791780E001C081E0DF91CF9108951092EE
:1021D000B9008CE08093B8000895EF92FF920F93BE
:1021E0001F93CF93DF93182FEB011092BC0084EA6A
:1021F0008093BC000E944F1F7C018091BC0087FD32
:102200000EC0CF3F8FEFD807C1F30E944F1F8E192A
:102210009F098C179D0788F38EEF9FEF2EC080914A
:10222000B900887F883041F08091B900887F803183
:1022300019F08FEF9FEF21C01093BB0084E88093CB
:10224000BC000E944F1F8C018091BC0087FD0CC018
:10225000CF3F8FEFD807C1F30E944F1F801B910B18
:102260008C179D0788F3D8CF8091B900887F88317B
:1022700011F08034F1F680E090E0DF91CF911F9172
:102280000F91FF90EF9008950F931F93CF93DF93DB
:10229000EB018093BB0084E88093BC000E944F1F39
:1022A0008C018091BC0087FD0EC0CF3F8FEFD80717
:1022B000C1F30E944F1F801B910B8C179D0788F361
:1022C0008EEF9FEF0CC02091B900287F81E090E055
:1022D000283211F480E090E0919581959109DF9189
:1022E000CF911F910F910895CF92DF92EF92FF92BD
:1022F0000F931F93CF93DF936B018A017901B9018B
:102300000E94ED10E6010C0D1D1DC017D10761F4F0
:1023100024E92093BC00DF91CF911F910F91FF9092
:10232000EF90DF90CF90089597FDF2CFB70189919C
:102330000E944411EACFCF92DF92EF92FF920F9367
:102340001F93CF93DF93C62F6A017901B8010E94D2
:10235000ED1097FD11C0B8018C2F0E944411E601C9
:10236000EC0CFD1CCE15DF0539F097FD05C0B8015A
:1023700089910E944411F6CF24E92093BC00DF919B
:10238000CF911F910F91FF90EF90DF90CF90089524
:1023900084E98093BC00089590937901809378013B
:1023A0000895E0917801F0917901309721F0019042
:1023B000F081E02D099480E00895E0917801F0919A
:1023C0007901309721F00280F381E02D099408957E
:1023D000E0917801F0917901309739F022E0DC0149
:1023E0002C930480F581E02D0994089520917601C5
:1023F000309177012817390771F090937701809316
:102400007601E0917801F0917901309721F0068012
:10241000F781E02D099408952091740130917501A0
:102420002817390771F09093750180937401E0913A
:102430007801F0917901309721F00084F185E02D49
:102440000994089585B7806885BF85B7806885BF82
:10245000089508950C9429120C942A120C942912B0
:102460000C9429120E9422120E942E120C942C12FB
:1024700081E008950E94461F0E94A80880E00E9403
:10248000690C0E94DB1F0E94EB090C9430129F9292
:10249000AF92BF92CF92DF92EF92FF920F931F9372
:1024A000CF93DF93CDB7DEB72A970FB6F894DEBF90
:1024B0000FBECDBF0E94F908C82E0E9438128111AC
:1024C00011C08FEF89838A831B820E944F1F816016
:1024D000782F9D838C8349815A816B818D810E94E5
:1024E000EA1240C08BE7A82E81E0B82E00E010E091
:1024F000902E802F0E949808E82EF501D1905F0160
:10250000D82631F40F5F1F4F0330110589F7D9CF5B
:102510008091D60181FD0E949E0880E0FF24F39403
:102520009D2D9F21D1F08E839F82EF2081E009F4C1
:1025300080E088870E944F1F8160782F9A87898763
:102540004E815F8168858A850E94EA12F801E5580C
:10255000FE4F8081F826F08205C08F5FFF0C83302C
:10256000F9F6D0CF0E94340B0E94D60EC1100E9403
:10257000A50D0E946D210E94D11190917A018917B9
:10258000B9F00E94D11180937A012A960FB6F8947F
:10259000DEBF0FBECDBFDF91CF911F910F91FF9096
:1025A000EF90DF90CF90BF90AF909F900C945A0522
:1025B0002A960FB6F894DEBF0FBECDBFDF91CF9144
:1025C0001F910F91FF90EF90DF90CF90BF90AF9051
:1025D0009F900895CF93DF93CDB7DEB72B970FB6BB
:1025E000F894DEBF0FBECDBF4F83588769877A87C7
:1025F0008B87DE01119686E0FD0111928A95E9F73D
:1026000085E0FE01379601900D928A95E1F74981A8
:102610005A816B817C818D819E810E94491A2B9603
:102620000FB6F894DEBF0FBECDBFDF91CF910895F6
:10263000FC01808191810E94A01C0895882309F4E7
:102640001AC18238C1F40E94D11181FD14C169E31D
:1026500080910801909109010E94B61E0E94201DE0
:102660002FEF81EE94E0215080409040E1F700C0D0
:10267000000069E319C08338F9F40E94D11180FD8C
:10268000FAC063E580910801909109010E94B61E8D
:102690000E94201D2FEF81EE94E021508040904059
:1026A000E1F700C0000063E5809108019091090105
:1026B0000E94B81E0C94201D8438C1F40E94D111D0
:1026C00082FDD9C067E480910801909109010E94C0
:1026D000B61E0E94201D2FEF81EE94E02150804015
:1026E0009040E1F700C0000067E4DECF9CEF980F58
:1026F000913A40F4682F80910801909109010E945D
:10270000B61ED8CF90E2980F983050F4877091E0C1
:1027100001C0990F8A95EAF7892F0E94E21CCACF5F
:102720009BE5980F933070F4853A29F0863A31F0A2
:1027300083E890E005C081E890E002C082E890E084
:102740000C94F61198E5980F973108F08EC0883AEE
:1027500009F445C0893A09F445C08A3A09F445C0EC
:102760008B3A09F445C08C3A09F445C08B3B09F417
:1027700045C08C3B09F445C08D3A09F445C0803B07
:1027800009F445C08E3A09F445C08F3A09F445C0B2
:10279000813B09F445C0823B09F445C0833B09F401
:1027A00045C0843B09F445C0853B09F445C0863BE0
:1027B00009F445C0873B09F445C0883B09F445C08E
:1027C000893B09F445C08D3B09F445C08E3B09F4B3
:1027D00045C08A3B09F445C080E090E044C082EEE9
:1027E00090E041C089EE90E03EC08AEE90E03BC0B0
:1027F00085EB90E038C086EB90E035C083EB90E04D
:1028000032C084EB90E02FC087EB90E02CC08CECC2
:1028100090E029C08DEC90E026C083E891E023C0D1
:102820008AE891E020C082E991E01DC084E991E04E
:102830001AC081E292E017C083E292E014C084E201
:1028400092E011C085E292E00EC086E292E00BC0F9
:1028500087E292E008C08FE690E005C080E790E054
:1028600002C08AE292E00C940C12803F20F00E9499
:1028700075200C9462210895882309F464C082387D
:1028800079F40E94D11181FF5EC069E38091080153
:10289000909109010E94B61E0E94201D69E310C09C
:1028A0008338B1F40E94D11180FF4DC063E580915F
:1028B0000801909109010E94B61E0E94201D63E547
:1028C00080910801909109010E94B81E0C94201D6E
:1028D000843879F40E94D11182FF35C067E4809179
:1028E0000801909109010E94B61E0E94201D67E414
:1028F000E7CF9CEF980F913A10F4682FE1CF90E268
:10290000980F983050F4877091E001C0990F8A9524
:10291000EAF7892F0E94E81CD9CF9BE5980F9330E6
:1029200020F480E090E00C94F61198E5980F973130
:1029300020F480E090E00C940C12803F20F00E9484
:10294000DD200C9462210895CF93C82F0E941E139E
:10295000C93349F42FEF87EE93E021508040904037
:10296000E1F700C000008C2FCF910C943C14882319
:1029700021F00E94E21C0C94201D0895882321F070
:102980000E94E81C0C94201D0895CF92DF92EF92D4
:10299000FF920F931F93CF93DF937C01062FC72FD6
:1029A000FC01158112951F70D281D1110E94FF1C6C
:1029B0000E94D81C882379F0DD2369F080E2800F23
:1029C000883048F082E00E946A1D0E94D81C91E085
:1029D000D82ED92601C0D12CCC2EC2948FE0C8228B
:1029E0008C2D90E08E30910508F00FC2FC01EA5A60
:1029F000FF4F0C948B298C2F807FCF70882311F090
:102A0000C295C07FDD2399F0CC2309F4C8C180E2D0
:102A1000800F883010F0011104C08C2F0E94E21C3E
:102A200003C08C2F0E94F21C0E94201DB8C1802F71
:102A30000E943C14CC2309F4E8C180E2800F883066
:102A400010F0011104C08C2F0E94E81C03C08C2FD1
:102A50000E94F81C0E94201DD8C18C2F807FCF704F
:102A6000803211F0C295C07F002319F00130C9F007
:102A700022C0DD2371F0112341F0113031F40E94A6
:102A8000051D8C2B0E940D1DC0C10E94051D8C2BA5
:102A90001DC0112319F0113009F4B7C10E94161D91
:102AA00025C0DD2321F0163008F0AFC10EC015306F
:102AB00008F0ABC11BC0DD2361F0112331F0F70139
:102AC000858180FF6CC18F7085838C2F0E94B71425
:102AD0009CC1112359F0093309F072C1FFEF17EEC1
:102AE00023E0F15010402040E1F768C18C2F0E9494
:102AF000BE148BC18C2F86958695837019F081301A
:102B000061F083C1DD2321F0802F9C2F937002C0E0
:102B100080E090E00E94F61180C1DD2321F0802F3B
:102B20009C2F937002C080E090E00E940C1275C14F
:102B3000DD23F9F0053F51F0063F71F0043FA9F4A1
:102B40008091FA039091FB0381600BC08091FA039E
:102B50009091FB03826005C08091FA039091FB0382
:102B600084609093FB038093FA03802F0E9475206A
:102B70001EC0053F51F0063F71F0043FA9F480915B
:102B8000FA039091FB038E7F0BC08091FA03909122
:102B9000FB038D7F05C08091FA039091FB038B7F2F
:102BA0009093FB038093FA03802F0E94DD200E9404
:102BB000622133C18C2F837009F047C0D11129C124
:102BC000202F229526952770220F220F602F6F70DD
:102BD000862F90E0A0E0B0E0022E04C0880F991F7D
:102BE000AA1FBB1F0A94D2F704FF10C04FE050E0A9
:102BF00060E070E004C0440F551F661F771F2A95E0
:102C0000D2F7409550956095709503C040E050E034
:102C1000BA01C695C695C3708A019B01082B192B72
:102C20002A2B3B2BC901B801C23049F058F4C130FE
:102C300019F00E941D1BEDC00E940B1BEAC00E94F0
:102C40002F1BE7C00E94091BE4C0DD2319F08C2F65
:102C5000817001C08695882309F4DBC0202F22955E
:102C600026952770220F220F602F6F70862F90E01D
:102C7000A0E0B0E0022E04C0880F991FAA1FBB1F5E
:102C80000A94D2F704FF10C04FE050E060E070E01B
:102C900004C0440F551F661F771F2A95D2F7409531
:102CA00050956095709503C040E050E0BA01C6951C
:102CB000C695C3708A019B01082B192B2A2B3B2B2D
:102CC000C901B801C23049F058F4C13019F00E946E
:102CD000E21B9FC00E94D01B9CC00E94F41B99C0A5
:102CE0000E94431B96C0CF70DD2339F08C2F0E94C9
:102CF000691B802F0E94B7148CC0802F0E94BE14C5
:102D00008C2F0E948A1B85C0023F01F128F4003FEE
:102D100041F0013FA1F03FC0033FF9F0043F39F11A
:102D20003AC0DD2341F0153008F06FC08C2F8F7151
:102D30000E94AF1B6AC0163008F067C0F7CFDD23D2
:102D400039F08C2F8F710E94691B5FC0DD23C9F39E
:102D50008C2F8F710E948A1B58C0DD2329F08C2F85
:102D60008F710E94541B51C00E944F1B4EC0DD2327
:102D700049F0CF718C2F0E94691B63E08C2F0E9459
:102D8000551D43C081E00E946A1D1230F0F182E0BF
:102D90000E946A1D3AC0DD2331F0112391F2802F89
:102DA0000E941E1332C0112399F2093349F41FEF18
:102DB00027EE33E0115020403040E1F700C0000022
:102DC000802F0E943C1421C0D11127C0CF70C23087
:102DD00091F038F4CC2361F0C130B9F40E942F0A8D
:102DE0001CC0C43071F050F0C53079F480E00AC0E6
:102DF0000E940C0A12C00E94760A0FC00E947D0A2F
:102E00000CC083E00E94BF0A08C088EF8C0D84309C
:102E100020F40E94D1110E945A05DD20C9F00E94C1
:102E2000D41C80FD15C0F70112820E94CE1C0E94A6
:102E3000691BC7010E9431170E94CE1CDF91CF9100
:102E40001F910F91FF90EF90DF90CF900C948A1B11
:102E5000DF91CF911F910F91FF90EF90DF90CF9076
:102E600008950F931F93CF93DF93EC01988189818D
:102E70002B813C81232B31F08F3F31F481E09F3F48
:102E800019F403C081E001C080E080FD13C0CE01D1
:102E90000E947305882371F0688179818A810E947C
:102EA000AB1C8C010E94061C0E94F71AB801CE01CF
:102EB0000E94C514DF91CF911F910F9108950E9438
:102EC000FF1C0E94021D0E94201D0E9408220E94D9
:102ED000622180E090E00E94F61180E090E00C9486
:102EE0000C1280910801909109010E94BA1E0C9465
:102EF0005F170E94EF1C0C947117E92FE295EF7099
:102F00004E2F50E0FA013297EE30F105B0F4EC5953
:102F1000FF4F0C948B29803F91F018F4883E68F4A1
:102F20000EC0843F51F40BC0883E48F0813F29F425
:102F300006C093FB882780F9089580E0089581E01A
:102F400008950E94A01C0E947D170895CF93DF93DF
:102F500000D000D01F92CDB7DEB70F900F900F902A
:102F60000F900F90DF91CF910895CF93DF9300D012
:102F700000D000D0CDB7DEB726960FB6F894DEBFEE
:102F80000FBECDBFDF91CF9108951F93CF93DF93F5
:102F9000C0917F0116E080918001C81799F0D0E0C0
:102FA0001C9FF0011D9FF00D1124EF57FE4F408133
:102FB000518162817381848195810E94B517219628
:102FC000C770E9CFDF91CF911F9108954091B10172
:102FD0005091B2016091B3017091B4018091B5013B
:102FE0009091B6010C94B517CF938091B60182955C
:102FF0008F7009F05FC08091B301882309F45AC033
:1030000080917F01B09180017091B101A091B201D6
:103010004091B4015091B50191E07F3F09F090E0FB
:10302000692FC6E08B1709F445C04115510521F001
:10303000AF3F21F020E003C021E001C0262F90E047
:1030400020FD35C0C89FF001C99FF00D1124EF5736
:10305000FE4F21812A132BC02081271328C02281F3
:10306000211125C0238134812417350710F4215004
:103070003109241B350B283C3105C8F42091B601D9
:103080002F7020612093B60126E0289FF001299F30
:10309000F00D1124EA57FE4F80818F70806180838C
:1030A00081EB91E00E943117CF910C94C5170196E6
:1030B0008770B8CFCF910895AF92BF92CF92DF9231
:1030C000EF92FF920F931F93CF93DF93CDB7DEB7AD
:1030D00061970FB6F894DEBF0FBECDBF8C0185E0BF
:1030E000F801DE011D9601900D928A95E1F7D80155
:1030F0004C9111965C9111971296EC903091B10120
:103100006091B2018091B4019091B501009731F0C6
:103110006F3F31F421E03F3F19F403C021E001C0CB
:1031200020E0B22FB170BB2E20FD60C1F801C3803A
:10313000D480A090B301AA2009F4EEC02091B6017A
:10314000C816D90628F0D601A81BB90BCD0104C0BA
:10315000809590958C0D9D1DFF24F394883C9105DE
:1031600080F0F12C207F09F09CC07C2DD98AC88A80
:103170006E2D89890E94A61781EB91E00E9431177C
:103180002DC1822F807F09F054C0561314C0431301
:1031900012C0FE2CE1100FC02F7020612093B601E9
:1031A0000E94E61781EB91E00E9431178091B601F1
:1031B000F80185835CC1CD2831F05F3F31F481E0B7
:1031C0004F3F19F403C081E001C080E080FD03C0DF
:1031D00081E08E2502C080E090E0F82FF170FF2E94
:1031E00080FF1CC080917F012091800136E0821712
:1031F00009F41AC190E0389FF001399FF00D1124B5
:10320000EF57FE4F6181561306C06081461303C01D
:103210006281E61203C001968770E9CFFE2CEE2092
:1032200009F425C18091B60181608093B601F12C2B
:103230001EC1561309C0431307C0E11005C0809199
:10324000B601F8018583A4C04D875E878D859E8574
:103250000E94A117882379F1EE2069F12091B6012F
:10326000822F82958F7090E0029774F08091B10167
:103270009091B20198878F831986DB86CA862C8746
:10328000CE0107960E94311786E0F801A1EBB1E06C
:1032900001900D928A95E1F70E94F4170E94E617BB
:1032A0000DC0561771F04D875E878D859E850E94F3
:1032B000A11781111AC0C8010E943117FF24F3948D
:1032C000D6C04313F0CFE110EECF8091B601F801E4
:1032D0008583C8010E94311786E0E1EBF1E0DF0150
:1032E0001D928A95E9F7FA2CC2C0EE2021F32091B5
:1032F000B601822F82958F7090E002972CF2809118
:10330000B1019091B2019A8389831B82DD82CC82C4
:103310002E83CE010196B6CFC816D90628F0F60145
:10332000E81BF90BCF0104C0809590958C0D9D1D75
:10333000883C910548F0F12C7C2DD98AC88A6E2DE5
:1033400089890E94A6174AC0FE2CEE2009F4B3CF4B
:10335000561333C0431331C02091B60120FD24C061
:10336000822F82958F70482F50E041155105E1F072
:10337000D80115962C9315974F30510549F08F5F62
:10338000982F9295907F822F8F70892B15968C9312
:10339000C8010E94311786E0F801A1EBB1E001906D
:1033A0000D928A95E1F73DC086E0F801A1EBB1E00E
:1033B00001900D928A95E1F75AC04D875E878D8501
:1033C0009E850E94A11781115FCF8091B601816017
:1033D0008093B601C8010E94311749C0E1EBF1E0CA
:1033E00086E0DF011D928A95E9F71BC0EE2009F403
:1033F00062CF4D875E878D859E850E94A117F82E2E
:10340000882309F458CF86E0F801A1EBB1E00190E0
:103410000D928A95E1F781EB91E00E9418130E94CA
:10342000F4170E94E61723C04D875E878D859E8521
:103430000E94A01C292F22952F70223028F49F7003
:1034400039F0811105C00BC0243028F49F7049F475
:10345000805E883020F0C8010E943117BF2CFB2C01
:1034600006C0D80115969C91907F91F7F8CF8F2DCB
:1034700061960FB6F894DEBF0FBECDBFDF91CF913E
:103480001F910F91FF90EF90DF90CF90BF90AF9082
:1034900008951F93CF93DF93CDB7DEB72C970FB668
:1034A000F894DEBF0FBECDBF4F83588769877A87F8
:1034B0008B879C87CE0107960E945C188823D1F0E9
:1034C0009F8188852A853B85232B31F08F3F31F4FE
:1034D00081E09F3F19F403C081E001C080E080FDDE
:1034E00047C04F81588569857A858B859C850E9468
:1034F000B5173EC086E0FE013796DE0111960190B9
:103500000D928A95E1F7FF81E8856A857B856115D3
:10351000710531F0EF3F31F481E0FF3F19F403C052
:1035200081E001C080E080FD23C02091800130E077
:10353000C90101968770992740917F0150E0841757
:103540009507F1F1F983EA837D836C8396E0929F7E
:10355000D001939FB00D1124AF57BE4FFE0131969D
:1035600001900D929A95E1F7809380010E94C51712
:1035700016E080917F0190918001891771F1189F69
:10358000C00111248F579E4F0E945C18882329F197
:10359000E0917F011E9FF0011124EF57FE4F408103
:1035A000518162817381848195810E94B5178091D8
:1035B0007F0190E001968770992780937F01D9CF92
:1035C0000E9479171092800110927F01E1EBF1E0E7
:1035D00086E0DF011D928A95E9F72C960FB6F894E4
:1035E000DEBF0FBECDBFDF91CF911F91089508952B
:1035F00008950C94F81A0C94F91A0E94FB1A60931F
:10360000C5017093C6018093C7019093C8010C94C3
:103610005F170C94FD1A0F931F930091C501109131
:10362000C6012091C7013091C801602B712B822BFC
:10363000932B1F910F910C94FD1A0F931F930091E0
:10364000C5011091C6012091C7013091C8016023C6
:103650007123822393231F910F910C94FD1A0F93D2
:103660001F930091C5011091C6012091C7013091AF
:10367000C80160277127822793271F910F910C940F
:10368000FD1A0C94F81A0E94411B6093C1017093BB
:10369000C2018093C3019093C4010C945F1760E052
:1036A00070E0CB010C94431B0F931F9341E050E05B
:1036B00060E070E08A019B0104C0000F111F221F0F
:1036C000331F8A95D2F7C901B8011F910F910C944D
:1036D000431B0F931F9341E050E060E070E004C093
:1036E000440F551F661F771F8A95D2F78091C1013D
:1036F0009091C201A091C301B091C4018A019B01C4
:10370000082B192B2A2B3B2BC901B8011F910F91B4
:103710000C94431B0F931F9341E050E060E070E076
:1037200004C0440F551F661F771F8A95D2F7409536
:103730005095609570958091C1019091C201A091C2
:10374000C301B091C4018A019B01082319232A23D4
:103750003B23C901B8011F910F910C94431B0F9398
:103760001F9341E050E060E070E004C0440F551F3B
:10377000661F771F8A95D2F78091C1019091C2018F
:10378000A091C301B091C4018A019B0108271927A8
:103790002A273B27C901B8011F910F910C94431BA5
:1037A0000F931F930091C1011091C2012091C30199
:1037B0003091C401602B712B822B932B1F910F91A1
:1037C0000C94431B0F931F930091C1011091C201F0
:1037D0002091C3013091C40160237123822393237C
:1037E0001F910F910C94431B0F931F930091C101E4
:1037F0001091C2012091C3013091C401602771274B
:10380000822793271F910F910C94431B0895292F12
:10381000220F920F890FE82FE695E695E6958770BF
:1038200051E001C0550F8A95EAF785E0E89FF00165
:103830001124E954FE4F20E030E070E04081CB01DC
:10384000022E02C0969587950A94E2F781708195C1
:1038500084278523842781932F5F3F4F25303105AF
:1038600069F70895292F220F920F890F682F669507
:1038700066956695982F977085E0689FB001112432
:1038800040E050E080E0FB01E40FF51FE954FE4FFB
:10389000208130E0092E02C0369527950A94E2F780
:1038A00021703327042E01C0220F0A94EAF7822BDD
:1038B0004F5F5F4F4530510531F70895BF92CF926A
:1038C000DF92EF92FF920F931F93CF93DF938C01C0
:1038D000C090C101D090C201E090C301F090C4013A
:1038E0008091C5019091C601A091C701B091C80116
:1038F000C82AD92AEA2AFB2ACFE1D0E0D701C6019B
:103900000C2E04C0B695A795979587950A94D2F783
:1039100080FD04C0219790F7B12C07C0BC2EB801E0
:103920008C2F0E94F5050197A9F38B2DDF91CF9184
:103930001F910F91FF90EF90DF90CF90BF9008956F
:10394000CF93DF93EC010E945E1CBE010E94F5053F
:10395000DF91CF9108951F93CF93DF93EB01909167
:103960007E01992321F0CB010E94A01C13C0882363
:1039700049F0CB010E945E1C182F682FCE010E94D7
:10398000071C04C0CB010E94321C182FBE01812FDE
:103990000E94F505DF91CF911F9108958091C90193
:1039A00085958595859508958091C90187700895BD
:1039B0009091C901977081E009F480E008958091A9
:1039C000D50108959091D501892B8093D501089553
:1039D00080959091D50189238093D5010895109207
:1039E000D50108959091D401892B8093D401089535
:1039F00080959091D40189238093D40108951092E9
:103A0000D40108951092D30108958091CA010895B8
:103A100008950C94081D0C94091D9091CA019817E3
:103A200021F08093CA010C940B1D08958091CA0166
:103A3000882329F01092CA0180E00C940B1D089590
:103A4000E0910801F09109018091D5018083E09116
:103A50000801F091090190818091D401892B808324
:103A6000E0910801F091090190818091D301892BA7
:103A700080838091CA01882381F0E0910801F09150
:103A800009019081892B808380910801909109011F
:103A90000E94831E81110E94161D80910801909141
:103AA00009010C94DD110C94081D98E0899F900188
:103AB0001124262B2093C9010E94691B8091C90102
:103AC0008595859585950C94531D1092C90180E0CC
:103AD0000C94531D2091C901809582238093C901C4
:103AE000982F977079F430E0482F082E000C550B72
:103AF0002417350739F08595859585950E948A1B91
:103B00000C94651D0895CF92DF92EF92FF926C01A5
:103B1000EE24FF24C114D104E104F10421F0C70113
:103B2000B60120E101C020E0C72ED82EE92EFF24E7
:103B3000C114D104E104F10419F0285FC701B601F2
:103B40006B017C0154E0F694E794D794C7945A959E
:103B5000D1F7C114D104E104F10419F02C5FC701BD
:103B6000B6016B017C0142E0F694E794D794C794C8
:103B70004A95D1F7C114D104E104F10419F02E5F84
:103B8000C701B601DC01CB01B695A795979587953E
:103B9000892B8A2B8B2B09F02F5F822FFF90EF90C0
:103BA000DF90CF90089580E090E00E94C92921E045
:103BB0008C3E9E4F09F020E0822F089582E090E035
:103BC0000C94C12983E090E00C94C129CF9384E048
:103BD00090E00E94C129C82F81E290E00E94C12993
:103BE0002C2F30E0A901582BCA01CF910895CF9313
:103BF000C92F682F84E090E00E94CF296C2F81E2CA
:103C000090E0CF910C94CF2986E090E00C94C129EC
:103C1000682F86E090E00C94CF29AB01BC018FE0C7
:103C200090E00C94E129AB01BC0183E190E00C949D
:103C3000E12960E070E0CB010C94131E60E070E0BD
:103C4000CB010E940D1E0C94191E6CEE7EEF80E0DD
:103C500090E00E94ED2960E082E090E00E94CF2990
:103C600060E083E090E00E94CF291092C50110929D
:103C7000C6011092C7011092C80160E084E090E094
:103C80000E94CF2960E081E290E00E94CF2960E0AD
:103C900085E090E00E94CF2960E086E090E00E94FD
:103CA000CF296FEF87E090E00E94CF2940E050E0FD
:103CB000BA0188E090E00E94E12960E08DE090E0A8
:103CC0000E94CF2940E050E0BA0188E190E00E94D4
:103CD000E12960E087E190E00E94CF2940E050E0D8
:103CE000BA018CE190E00E94E12960E080E290E07E
:103CF0000E94CF290C941E1E0C94251E682F8EE066
:103D000090E00C94CF29FC01329697E080E091502E
:103D100029F021912223D9F38F5FF9CF08959C01D7
:103D2000FC0132969FEF80E04191461789F09F3F5A
:103D300019F4411101C0982F8F5F8630A9F79F3F7A
:103D400039F0F901E90FF11D97FDFA9562830895A5
:103D500008959C012A5F3F4FFC014281461301C038
:103D60001282019682179307B9F708950C948F1E5B
:103D70000C94A91E029626E0FC0111922A95E9F7FF
:103D8000089508950C94C11E0C94C11ECF930E94F7
:103D9000C41E0E94F9080E94C21EC0E08C2F0E941F
:103DA0009808811104C0CF5FC330C1F701C081E022
:103DB000CF9108950C94C11E0C94DA1E0E94DC1E53
:103DC00080910604843061F11092D70120E488E1EB
:103DD00090E00FB6F894A895809360000FBE2093F2
:103DE000600080E00E94120B80E00E945A050E9451
:103DF000DC1E83B7817F846083BF83B7816083BF0C
:103E00007894889583B78E7F83BF0FB6F894A89572
:103E100080916000886180936000109260000FBE06
:103E200008950C94C11E0E9479170E94EB090E940C
:103E3000D1110E945A050C94111F1F920F920FB6B8
:103E40000F9211248F939F93AF93BF938091D701CB
:103E5000811113C08091FC039091FD03A091FE039A
:103E6000B091FF034196A11DB11D8093FC03909377
:103E7000FD03A093FE03B093FF03BF91AF919F9109
:103E80008F910F900FBE0F901F90189582E084BD08
:103E900093E095BD9AEF97BD80936E0008952FB77C
:103EA000F8948091FC039091FD03A091FE03B091E2
:103EB000FF032FBF08952FB7F8946091FC03709112
:103EC000FD038091FE039091FF032FBF0895CF92D1
:103ED000DF92EF92FF920F931F932FB7F8944091C8
:103EE000FC035091FD036091FE037091FF032FBF0F
:103EF0006A017B01EE24FF248C0120E030E0C01633
:103F0000D106E206F30610F4415051099A01281B2C
:103F1000390BC9011F910F91FF90EF90DF90CF9067
:103F2000089578941F920F920FB60F9211248F93D9
:103F30009F93AF93BF938091FC039091FD03A09159
:103F4000FE03B091FF030196A11DB11D8093FC03F8
:103F50009093FD03A093FE03B093FF03BF91AF9135
:103F60009F918F910F900FBE0F901F90189581E039
:103F70008093E00080E28093D8001092C9008FE126
:103F80009EE40197F1F700C0000087E090EBDC01B0
:103F900080930F0490931004A0931104B093120423
:103FA0009CE088E10FB6F894A895809360000FBE5E
:103FB00090936000FFCF0E94D31D811102C00E9428
:103FC0007C1E0E94DE1D8093D6010E94E61D909308
:103FD0000104809300040E94E21D682F70E080E0DD
:103FE00090E00C94091B8091DB0180FF0BC0609175
:103FF0000D0185E0689FB001112475956795759551
:1040000067952BC081FF09C060910D0185E0689F15
:10401000B00111247595679520C082FF07C060919B
:104020000D0185E0689FB001112417C09091DA015D
:104030009923D1F060910C01961788F720910D011A
:1040400085E0289F90011124929FA001939F500D1D
:10405000112470E0CA010E9455296038710540F4AE
:104060006115710519F406C065E070E0862F0895AA
:104070008FE7089581E008958091DB0180FF08C0FB
:1040800060910B0170E0759567957595679521C0F6
:1040900081FF06C060910B0170E07595679519C0AE
:1040A00082FF04C060910B0170E010C09091DA01B2
:1040B000992399F060910A019617A0F780910B015E
:1040C000899FC001112470E00E9455296038710554
:1040D00040F46115710519F406C061E070E0862FA7
:1040E00008958FE7089581E00895803F21F40E94AC
:1040F000F31F819504C0813F29F40E94F31F809330
:10410000DF010895823F21F40E94F31F819504C0CE
:10411000833F29F40E94F31F8093DE010895893FB5
:1041200019F40E943C2005C08A3F31F40E943C20D3
:1041300081958093E00108958B3F21F40E943C20FB
:10414000819504C08C3F29F40E943C208093E101BA
:104150000895843F21F48091DD01816017C0853F7F
:1041600021F48091DD01826011C0863F21F48091AD
:10417000DD0184600BC0873F21F48091DD01886000
:1041800005C0883F31F48091DD0180618093DD01BD
:1041900008958D3F21F48091DB0181600BC08E3F3B
:1041A00021F48091DB01826005C08F3F29F480916A
:1041B000DB0184608093DB010895803F39F48091B6
:1041C000DF0187FF6CC01092DF0169C0813F29F4D5
:1041D0008091DF011816BCF362C09091DE01823F2E
:1041E00029F497FF5CC01092DE0159C0833F19F497
:1041F0001916CCF354C0893F41F48091E0011816A0
:104200000CF04DC01092E0014AC08A3F29F4809121
:10421000E00187FF44C0F6CF8B3F39F48091E10184
:1042200087FF3DC01092E1013AC08C3F29F4809194
:10423000E1011816BCF333C0843F21F48091DD0105
:104240008E7F17C0853F21F48091DD018D7F11C0E5
:10425000863F21F48091DD018B7F0BC0873F21F4E5
:104260008091DD01877F05C0883F31F48091DD01B9
:104270008F7E8093DD0113C08D3F21F48091DB019F
:104280008E7F0BC08E3F21F48091DB018D7F05C0B6
:104290008F3F29F48091DB018B7F8093DB0180913C
:1042A000DE0181110EC08091DF0181110AC0809171
:1042B000E001811106C08091E101811102C01092DC
:1042C000DA0108958CED91E00E94E8110E944F1FE1
:1042D0009093D9018093D80108951F93CF93DF93D2
:1042E0008091D8019091D9010E94671FAC019091F3
:1042F000DA01992321F020910E0130E006C02091CF
:104300000F018AE0289F900111244217530708F4F7
:104310007BC08091DE01C091DF01D091E00110915E
:10432000E101811107C0C1116BC0D11169C0111128
:1043300067C06AC09F3F19F09F5F9093DA0118161B
:1043400024F40E94F31F8093DE018091DE0187FF39
:1043500005C00E94F31F81958093DE011C1624F492
:104360000E94F31F8093DF018091DF0187FF05C06A
:104370000E94F31F81958093DF013091DE0133238A
:10438000E1F02091DF012223C1F045EB3403C001AD
:104390001124992319F09093DE0103C081E08093EA
:1043A000DE0135EB2303C0011124992319F090930A
:1043B000DF0103C081E08093DF011D1624F40E9419
:1043C0003C208093E0018091E00187FF05C00E94BE
:1043D0003C2081958093E001111624F40E943C203A
:1043E0008093E1018091E10187FF05C00E943C209C
:1043F00081958093E101DF91CF911F910C9462210F
:104400009F3F09F099CFAACFDF91CF911F910895D7
:10441000ECEDF1E086E0DF011D928A95E9F710925C
:10442000DA011092DB0108958091EA0108950F935B
:104430001F93CF93DF9300D01F92CDB7DEB78C01CF
:104440000E946A24823011F0843021F584E089834F
:104450001B830A8382E08093E9008FEF9091E8004C
:10446000815095FD06C095ED9A95F1F700008111F8
:10447000F5CF8091E80085FF0DC040E050E063E09B
:1044800070E0CE0101960E9487248091E8008E772B
:104490008093E8000F900F900F90DF91CF911F91C4
:1044A0000F910895CF93DF9300D01F92CDB7DEB761
:1044B00020910604243031F523E0298380589109A6
:1044C0009B838A8382E08093E9008FEF9091E800DC
:1044D000815095FD06C095ED9A95F1F70000811188
:1044E000F5CF8091E80085FF0DC040E050E063E02B
:1044F00070E0CE0101960E9487248091E8008E77BB
:104500008093E8000F900F900F90DF91CF91089566
:10451000CF93DF93EC010E946A24823011F0843043
:10452000F9F482E08093E9008FEF9091E8008150E8
:1045300095FD06C095ED9A95F1F700008111F5CF34
:104540008091E80085FF0CC040E050E066E070E03C
:10455000CE010E9487248091E8008E778093E80046
:10456000DF91CF910895CF93DF93EC010E946A24ED
:10457000823011F0843039F581E08093E9008FEFCB
:104580009091E800815095FD06C095ED9A95F1F760
:1045900000008111F5CF8091E80085FF14C040E054
:1045A00050E068E070E0CE010E9487248091E8002E
:1045B0008E778093E80088E0FE01A2EEB1E00190E2
:1045C0000D928A95E1F7DF91CF91089580910504CE
:1045D000811109C00E9418260E9475268091E20070
:1045E00084608093E2000895109205040895089570
:1045F00008950C94131F42E061EC81E00E94912524
:1046000042E261EC82E00C949125809108048330B1
:1046100009F460C030F4813071F0823009F499C03F
:1046200008958A3009F485C08B3009F46BC0893055
:1046300009F0A7C020C080910704813A09F0A1C009
:104640008091E800877F8093E80080910B0490912F
:104650000C04892B21F468E082EE91E003C060E055
:1046600080E090E070E00E94D2248091E8008B7797
:104670008093E800089580910704813209F081C099
:1046800080910B0490910C04029708F07AC08091FD
:10469000E800877F8093E8008091E80082FD05C0F4
:1046A000809106048111F8CF6CC02091F3008091B5
:1046B000F20090E0922B029729F48091F1008B7F19
:1046C000813021F48091F1008093EA018091E8002B
:1046D0008B7753C080910704813A09F052C08091D2
:1046E0000B0490910C04892B09F04BC08091E800D9
:1046F000877F8093E8008091E80080FFFCCF809165
:104700001A0136C0809107048132D9F580910B04DB
:1047100090910C04892BA9F58091E800877F809304
:10472000E8000E94C6258091090480931A010C9428
:10473000791780910704813221F58091E800877F05
:104740008093E8000E94C62580910A048093EB01C3
:10475000089580910704813AA1F48091E800877F51
:104760008093E8008091E80080FFFCCF8091EB010E
:104770008093F1008091E8008E778093E8000C949C
:10478000C625089584B7877F84BF0FB6F894A8958F
:1047900080916000886180936000109260000FBE7D
:1047A00090E080E80FB6F8948093610090936100E8
:1047B0000FBE0E9432120E9418260E947526809118
:1047C000E20084608093E20078940E940A290E94AB
:1047D0003A1280E191E00E94CC118091060485306C
:1047E00069F40E94DE1E809104048823B1F30E94C4
:1047F000C61E882391F30E947124EFCF0E944712B6
:10480000ECCF0C940324292F332723303105C9F032
:1048100060F42130310581F02230310509F04AC0C1
:104820008BE390E027E937E049C02132310511F1EF
:104830002232310579F13EC082E190E022ED37E08D
:104840003DC099278130910561F040F0823091059B
:1048500059F0039779F5EFE4F7E008C0E3E9F7E0F2
:1048600005C0EFE7F7E002C0E5E5F7E0849190E0EE
:104870009F0124C06115710541F061307105D1F4CB
:1048800089E090E022EC37E019C089E090E029EA65
:1048900037E014C06115710541F06130710551F4C4
:1048A00085E890E024EE37E009C080E490E029E656
:1048B00038E004C080E090E020E030E0FA0131838D
:1048C0002083089580910604843011F081E00895DA
:1048D00082E008958091EC01811102C00C94622461
:1048E000089580E189BD82E189BD09B400FEFDCF54
:1048F0008091D8008F7D8093D8008091E000826005
:104900008093E0008091E00081FDFCCF0895CF927C
:10491000DF92EF92FF920F931F93CF93DF93EC01FF
:104920008B017A010E94E525811133C0E114F10465
:1049300039F0F70180819181081B190BC80FD91F2D
:10494000C12CD12C0115110519F18091E80085FDCC
:1049500016C08091E8008E778093E800E114F1049E
:1049600049F0F70180819181C80ED91ED182C082A1
:1049700085E00FC00E94E525882321F30AC08991B4
:104980008093F10001501109FFEFCF1ADF0ADACF4F
:1049900080E0DF91CF911F910F91FF90EF90DF901A
:1049A000CF90089520910D0430910E0426173707FB
:1049B00048F06115710539F42091E8002E772093B5
:1049C000E80001C0B901FC0120E06115710579F131
:1049D000809106048823F1F18530F1F18091E8009F
:1049E00083FD3CC08091E80082FD2EC08091E800EC
:1049F00080FFEBCF2091F3008091F20090E0922BAA
:104A00006115710551F08830910538F4219120939A
:104A1000F100615071090196F3CF21E0089709F088
:104A200020E08091E8008E778093E800CECF2111BE
:104A3000CFCF0AC080910604882361F0853061F0F1
:104A40008091E80083FD0AC08091E80082FFF2CFE8
:104A500080E0089582E0089583E0089581E008955C
:104A600020910D0430910E042617370748F0611588
:104A7000710539F42091E8002E772093E80001C0F9
:104A8000B901FC0120E06115710591F180910604E6
:104A9000882309F440C0853009F43FC08091E800C4
:104AA00083FD3DC08091E80082FD2FC08091E80029
:104AB00080FFE9CF2091F3008091F20090E0922BEB
:104AC0006115710559F08830910540F424912093C7
:104AD000F1003196615071090196F2CF21E00897FB
:104AE00009F020E08091E8008E778093E800CBCF3A
:104AF0002111CCCF0AC080910604882361F0853053
:104B000061F08091E80083FD0AC08091E80082FF97
:104B1000F2CF80E0089582E0089583E0089581E077
:104B20000895982F973068F59093E900981739F019
:104B30007091EC002091ED005091F00003C0242F03
:104B4000762F50E021FD02C09F5FECCF3091EB004B
:104B50003E7F3093EB003091ED003D7F3093ED00D0
:104B60003091EB0031603093EB007093EC002093B8
:104B7000ED005093F0002091EE0027FDE5CF80E09E
:104B800008958F708093E90081E008958091070473
:104B900087FF11C08091E80082FD05C08091060466
:104BA0008111F8CF11C08091E8008B770BC0809104
:104BB0000604882349F08091E80080FFF8CF8091B7
:104BC000E8008E778093E80008952091E40030910A
:104BD000E50095E64091EC00842F817040FF23C0F2
:104BE0008091E80080FD1DC080910604882399F023
:104BF000853099F08091EB0085FD11C04091E40073
:104C00005091E5002417350729F3915011F09A01CE
:104C1000E1CF84E0089582E0089583E0089581E083
:104C2000089580E008954091E80042FFDDCF0895A7
:104C30000E9486260E948E26E0EEF0E08081816050
:104C40008083E8EDF0E080818F77808319BCA7ED49
:104C5000B0E08C918E7F8C9380818F7E80831092C8
:104C6000050408950F931F93CF93DF930E94862628
:104C70000E948E26C8EDD0E088818F778883888156
:104C80008068888388818F7D888319BC1092060490
:104C900010920204109204041092030400EE10E03B
:104CA000F80180818B7F808388818160888342E0E6
:104CB00060E080E00E949125E1EEF0E080818E7F4F
:104CC0008083E2EEF0E08081816080838081886073
:104CD0008083F80180818E7F8083888180618883D2
:104CE000DF91CF911F910F910895E8EDF0E0808161
:104CF0008F7E8083E7EDF0E080818160808384E0B7
:104D000082BF81E0809305040C943226E8EDF0E048
:104D100080818E7F80831092E20008951092DA00E5
:104D20001092E10008951F920F920FB60F92112476
:104D30002F933F934F935F936F937F938F939F93A3
:104D4000AF93BF93EF93FF938091E10082FF0BC07D
:104D50008091E20082FF07C08091E1008B7F809309
:104D6000E1000E9409298091DA0080FF1FC0809134
:104D7000D80080FF1BC08091DA008E7F8093DA001C
:104D80008091D90080FF0DC080E189BD82E189BD9D
:104D900009B400FEFDCF81E0809306040E94E62264
:104DA00005C019BC109206040E94F4228091E10013
:104DB00080FF19C08091E20080FF15C08091E20061
:104DC0008E7F8093E2008091E20080618093E20018
:104DD0008091D80080628093D80019BC85E08093D0
:104DE00006040E94F8228091E10084FF30C0809187
:104DF000E20084FF2CC080E189BD82E189BD09B455
:104E000000FEFDCF8091D8008F7D8093D8008091E7
:104E1000E1008F7E8093E1008091E2008F7E80939D
:104E2000E2008091E20081608093E20080910204C0
:104E3000882311F084E007C08091E30087FD02C061
:104E400081E001C083E0809306040E94F9228091F2
:104E5000E10083FF29C08091E20083FF25C080919B
:104E6000E100877F8093E10082E080930604109246
:104E700002048091E1008E7F8093E1008091E20046
:104E80008E7F8093E2008091E20080618093E20057
:104E900042E060E080E00E9491258091F00088600F
:104EA0008093F0000E94F722FF91EF91BF91AF91A4
:104EB0009F918F917F916F915F914F913F912F9132
:104EC0000F900FBE0F901F9018951F920F920FB664
:104ED0000F9211242F933F934F935F936F937F9380
:104EE0008F939F93AF93BF93CF93DF93EF93FF93F2
:104EF000C091E900CF708091EC00D82FD17080FD77
:104F0000D0E81092E9008091F000877F8093F00054
:104F100078940E94A9271092E9008091F00088609F
:104F20008093F000CD2BCF70C093E900FF91EF91FB
:104F3000DF91CF91BF91AF919F918F917F916F91B1
:104F40005F914F913F912F910F900FBE0F901F9047
:104F500018951F93CF93DF93CDB7DEB7AA970FB6FF
:104F6000F894DEBF0FBECDBFE7E0F4E08091F10022
:104F7000819324E0EF30F207C9F70E940523809166
:104F8000E80083FF2EC18091070490910804492F07
:104F900050E04A30510508F024C1FA01EE58FF4FA5
:104FA0000C948B29803821F0823809F01AC108C08E
:104FB0008091030490910404992389F082600FC0CA
:104FC00080910B048F70873008F00BC18093E9004B
:104FD0008091EB0085FB882780F91092E900909181
:104FE000E800977F9093E8008093F1001092F10021
:104FF000D1C0282F2D7F09F0F4C0882319F082300A
:1050000061F0EFC080910904813009F0EAC093306B
:1050100009F080E0809304042EC08091090481117E
:105020002AC080910B048F702FEF280F263008F0D4
:10503000D8C08093E9002091EB0020FF1CC0933082
:1050400021F48091EB00806214C09091EB0090619C
:105050009093EB0021E030E0A90102C0440F551FFE
:105060008A95E2F74093EA001092EA008091EB0003
:1050700088608093EB001092E9008091E800877FC0
:105080008093E8000E94C625ACC08111AAC010918F
:1050900009041F778091E3008078812B8093E300DF
:1050A0008091E800877F8093E8000E94C625809168
:1050B000E80080FFFCCF8091E30080688093E300EC
:1050C000111102C082E001C083E08093060489C010
:1050D0008058823008F085C08091090490910A04BC
:1050E0008C3D53E0950779F583E08A838AE28983D2
:1050F0004FB7F894DE01139620E03EE051E2E32F33
:10510000F0E050935700E49120FF03C0E295EF7068
:105110003F5FEF708E2F90E0EA3010F0C79601C02D
:10512000C0968D939D932F5F243149F74FBF809197
:10513000E800877F8093E8006AE270E0CE01019684
:105140000E94D22416C060910B0470910C04AE0131
:105150004F5F5F4F0E940124BC01892B09F441C0BD
:105160009091E800977F9093E80089819A810E944E
:1051700030258091E8008B778093E80032C080383A
:1051800081F58091E800877F8093E8008091020498
:105190008093F1008091E8008E7772CF811121C059
:1051A0008091090490910A0499270297D4F4809180
:1051B000E800877F8093E8008091090480930204CF
:1051C0000E94C62580910204811106C08091E300EF
:1051D00087FD02C081E001C084E0809306040E9444
:1051E000FB228091E80083FF0AC08091E800877F5E
:1051F0008093E8008091EB0080628093EB00AA9698
:105200000FB6F894DEBF0FBECDBFDF91CF911F91D7
:1052100008950895CF93809106048823A1F0C0914A
:10522000E900CF709091EC00892F817090FD80E8AB
:10523000C82B1092E9008091E80083FD0E94A92705
:10524000CF70C093E900CF910895DB018F939F93B6
:105250000E94A029BF91AF91A29F800D911DA39F95
:10526000900DB29F900D11240895991B79E004C010
:10527000991F961708F0961B881F7A95C9F7809595
:105280000895AA1BBB1B51E107C0AA1FBB1FA6178D
:10529000B70710F0A61BB70B881F991F5A95A9F7DF
:1052A00080959095BC01CD01089597FB072E16F4CB
:1052B000009407D077FD09D00E94412907FC05D052
:1052C0003EF4909581959F4F0895709561957F4F1D
:1052D0000895A1E21A2EAA1BBB1BFD010DC0AA1F37
:1052E000BB1FEE1FFF1FA217B307E407F50720F04F
:1052F000A21BB30BE40BF50B661F771F881F991FCA
:105300001A9469F760957095809590959B01AC0112
:10531000BD01CF010895EE0FFF1F0590F491E02D20
:105320000994A29FB001B39FC001A39F700D811D7E
:105330001124911DB29F700D811D1124911D08959E
:105340000E949129A59F900DB49F900DA49F800D60
:10535000911D11240895FB01DC0102C005900D92FE
:1053600041505040D8F70895FB01DC0104C08D91F5
:105370000190801921F441505040C8F7881B990BC7
:105380000895F999FECF92BD81BDF89A992780B50D
:105390000895A8E1B0E042E050E00C94F529262FF2
:1053A000F999FECF92BD81BDF89A019700B402161B
:1053B00039F01FBA20BD0FB6F894FA9AF99A0FBEC9
:1053C00008950396272F0E94D0290E94CF29252FC8
:1053D0000E94D029242F0C94D0290196272F0E94B7
:1053E000D0290C94CF29DC01CB01FC01F999FECF27
:1053F00006C0F2BDE1BDF89A319600B40D9241505D
:0A5400005040B8F70895F894FFCF6C
:10540A00060021007F220003CB012808140A321E5D
:10541A001422B32288225222172201F73133F4F5DB
:10542A00F600FF0100010000FFFF0000010001FF7C
:0A543A000000081018181008000008
:00000001FF
